:100000000C943E000C945B000C945B000C945B0021
:100010000C945B000C945B000C945B000C945B00F4
:100020000C945B000C945B000C945B000C945B00E4
:100030000C945B000C945B000C945B000C945B00D4
:100040000C945B000C945B000C945B000C945B00C4
:100050000C945B000C945B000C945B000C945B00B4
:100060000C945B000C945B000C945B000C945B00A4
:100070000C945B000C945B000C945B0011241FBE7D
:10008000CFEFD8E0DEBFCDBF11E0A0E0B1E0E4E10A
:10009000F5E002C005900D92A231B107D9F711E049
:1000A000A2E1B1E001C01D92AA32B107E1F70E94BE
:1000B0000B010C9489020C940000409110015091A6
:1000C000110120E030E0682F772702C02F5F3F4FFB
:1000D00080B19927807190708617970719F02417BF
:1000E0003507A1F780E090E02417350711F481E08F
:1000F00090E00895409110015091110120E030E00E
:10010000682F772702C02F5F3F4F80B199278870F3
:1001100090708617970719F024173507A1F780E02C
:1001200090E02417350711F481E090E008950F93D3
:100130001F930B980C9800E010E080E00E945D0097
:100140008823F9F406950399006880E10E945D0018
:100150008823B9F41F5F183081F788E00E947A0085
:10016000882379F40B9A139820E0E5E0F0E0CF01C2
:100170000197F1F72F5F2431D1F70B98802F992742
:1001800002C080E090E01F910F9108950F931F939C
:10019000182F0C980B9A139880E00E945D0088231A
:1001A00019F08FEF90E02DC000E010FF02C0139A0D
:1001B00001C0139880E10E945D008823D1F40E9461
:1001C0005D008823C9F40F5F083011F01695EDCF5C
:1001D0000B9880E00E947A00882319F08CEF90E061
:1001E00010C080E10E945D00882349F08BEF90E011
:1001F00008C08EEF90E005C08DEF90E002C080E077
:1002000090E01F910F910895FC0180819927089536
:10021000FC016083089514BE80E18093600041E09A
:100220003FEFA8E8B3E14093290131B9809129015A
:1002300082B920E0CD010197F1F72F5F2436D1F785
:1002400080912901880F80932901809129018823B9
:1002500061F731B912B8409329015FEFE8E8F3E1A3
:1002600054B98091290185B920E0CF010197F1F7B8
:100270002F5F2436D1F780912901880F80932901BF
:1002800080912901882361F734B915B84093290179
:100290005FEFE8E8F3E157B98091290188B920E0E0
:1002A000CF010197F1F72F5F2436D1F78091290113
:1002B000880F8093290180912901882361F737B93C
:1002C00018B8409329015FEFE8E8F3E15AB980914B
:1002D00029018BB920E0CF010197F1F72F5F243678
:1002E000D1F780912901880F8093290180912901FC
:1002F000882361F73AB91BB896CFDF92EF92FF924D
:100300000F931F93CF93DF93EC010C980B9A1398E4
:1003100080911201049B04C084608093120106C086
:100320008B7F80931201882309F4EBC0F894282F67
:100330003327E1E0DE2ED22221FF0EC0E0E0F1E023
:1003400080819181C817D90711F442E0D42A3296EE
:1003500081E0E031F807A1F722FF03C0E4E0DE2AE4
:1003600003C0DD2009F4CAC00B9880E10E945D0043
:10037000882309F0C6C00E945D00882309F0C1C02F
:1003800080E10E945D00882309F0BBC080911201CA
:100390000E94C6008111DD248C2F0E94C6008111AD
:1003A000DD248D2F992787FD9A950E94C60088230A
:1003B00009F4A1C0DD249FC00E949700843809F48D
:1003C0006EC0853870F48138E1F0823820F48038CE
:1003D00009F091C013C08238C1F1833809F08BC095
:1003E0005AC0863809F463C0863808F45CC0873880
:1003F00009F463C0883809F07EC06DC00B9A139869
:100400007DC00E949700C82FDD270E949700992782
:10041000382F2227E0E0A0E0B1E004C0EF5F1296A1
:10042000E83069F18D919C9111978F5F9F4FB1F7E3
:10043000FF27EE0FFF1FE050FF4FC22BD32BD183BE
:10044000C08380E00E94C60056C00E949700082F1B
:1004500011270E9497009927382F2227202B312B14
:10046000E0E0A0E0B1E004C0EF5F1296E83039F0C0
:100470008D919C91119782179307B1F702C08FEF6E
:10048000E1CFFF27EE0FFF1FE050FF4F8FEF9FEFF1
:1004900091838083D6CF8091120182600BC08091BE
:1004A00012018D7F07C080911201816003C080918D
:1004B00012018E7F809312011EC00E949700082FA8
:1004C00011270E9497009927982F8827082B192B0E
:1004D000F8018081B7CF0E949700082F11270E9452
:1004E0009700E82E0E949700FF24FE2CEE240E2990
:1004F0001F29F8018083DD2009F05ECF0B9A139845
:100500007894DF91CF911F910F91FF90EF90DF9042
:040510000895FFCF7C
:10051400FFFFFFFFFFFFFFFFFFFFFFFFFFFFFFFFE7
:02052400307530
:00000001FF
